:020000040000FA
:04000000EFEF0AF024
:06002A00D9CFE5FFE1CF94
:10003000D9FF00C0E5FF01C0E5FF02C0E5FF03C036
:10004000E5FF04C0E5FF05C0E5FF06C0E5FF07C00A
:10005000E5FF08C0E5FF09C0E5FF0AC0E5FF020EA5
:10006000DBCF00F0030EDBCF01F0040EDBCF02F09C
:10007000050EDBCF03F0060EDBCF04F0070EDBCF5F
:1000800005F000C006F001C007F002C008F0035000
:1000900003E003500508036E270EE56E100EE56EB3
:1000A0000550E56E0450E56ED9EC05F0096EF3CF0E
:1000B0000AF0040EE126300E092609C0E5FF06C04D
:1000C000E9FF07C0F3FF0850FBEC0AF0062AD8B09E
:1000D000072AD8B0082A030603500EE12E0EE56E5B
:1000E00006C0E9FF07C0F3FF0850FBEC0AF0062A40
:1000F000D8B0072AD8B0082A270EE56E100EE56E94
:100100000550E56E0450E56E7DEC05F0046EF3CF0E
:1001100005F0040EE126030EE56EE80EE56E0550CF
:10012000E56E0450E56ED9EC05F0096EF3CF0AF0E8
:10013000040EE126300E092609C0E5FF06C0E9FFDE
:1001400007C0F3FF0850FBEC0AF0062AD8B0072AD4
:10015000D8B0082A030603500EE12E0EE56E06C045
:10016000E9FF07C0F3FF0850FBEC0AF0062AD8B0FD
:10017000072AD8B0082A030EE56EE80EE56E055092
:10018000E56E0450E56E7DEC05F0046EF3CF05F0EE
:10019000040EE126000EE56E640EE56E0550E56E78
:1001A0000450E56ED9EC05F0096EF3CF0AF0040EA9
:1001B000E126300E092609C0E5FF06C0E9FF07C0A9
:1001C000F3FF0850FBEC0AF0062AD8B0072AD8B093
:1001D000082A030603500EE12E0EE56E06C0E9FF65
:1001E00007C0F3FF0850FBEC0AF0062AD8B0072A34
:1001F000D8B0082A000EE56E640EE56E0550E56E77
:100200000450E56E7DEC05F0046EF3CF05F0040EAE
:10021000E126000EE56E0A0EE56E0550E56E04500F
:10022000E56ED9EC05F0096EF3CF0AF0040EE12675
:10023000300E092609C0E5FF06C0E9FF07C0F3FF3D
:100240000850FBEC0AF0062AD8B0072AD8B0082AD2
:10025000030603500EE12E0EE56E06C0E9FF07C04F
:10026000F3FF0850FBEC0AF0062AD8B0072AD8B0F2
:10027000082A000EE56E0A0EE56E0550E56E045084
:10028000E56E7DEC05F0046EF3CF05F0040EE1267B
:10029000300E042604C0E5FF06C0E9FF07C0F3FFE7
:1002A0000850FBEC0AF0062AD8B0072AD8B0082A72
:1002B000032E09D02E0EE56E06C0E9FF07C0F3FF3E
:1002C0000850FBEC0AF00050040F036E000E0120F2
:1002D000046E000E0220056E0250800FF36E055072
:1002E000800FF35C05E10450015C02E10350005C07
:1002F00019E200C0E9FF01C0F3FF0250A4EC0AF0CC
:10030000066E300A0FE1200EE56E00C0E9FF01C065
:10031000F3FF0250FBEC0AF0002AD8B0012AD8B053
:10032000022ADAD7E4CF0AF0E4CF09F0E4CF08F0EC
:10033000E4CF07F0E4CF06F0E4CF05F0E4CF04F01B
:10034000E4CF03F0E4CF02F0E4CF01F0E4CF00F01B
:10035000E4CFD9FF1200D9CFE5FFE1CFD9FF00C02C
:10036000E5FF01C0E5FF02C0E5FF03C0E5FF04C0F3
:10037000E5FF05C0E5FF06C0E5FF07C0E5FF020E8B
:10038000DBCF00F0030EDBCF01F0040EDBCF02F079
:10039000050EDBCF03F0640EE56E03C0E5FFF6EC5F
:1003A00008F0046EE450E450300E042604C0E5FF6B
:1003B00000C0E9FF01C0F3FF0250FBEC0AF000505F
:1003C000010F046E000E0120056E000E0220066E65
:1003D000640EE56E03C0E5FF4CEC08F0036EE450DC
:1003E000E4500A0EE56E03C0E5FFF6EC08F0076E78
:1003F000E450E450300E072607C0E5FF04C0E9FFD3
:1004000005C0F3FF0650FBEC0AF0042AD8B0052A19
:10041000D8B0062A0A0EE56E03C0E5FF4CEC08F0E2
:10042000036EE450E450300E032603C0E5FF04C021
:10043000E9FF05C0F3FF0650FBEC0AF00050020F85
:10044000036E000E0120046E000E0220056E0250A5
:10045000800FF36E0550800FF35C05E10450015CE2
:1004600002E10350005C19E200C0E9FF01C0F3FFA4
:100470000250A4EC0AF0066E300A0FE1200EE56E81
:1004800000C0E9FF01C0F3FF0250FBEC0AF0002AB4
:10049000D8B0012AD8B0022ADAD7E4CF07F0E4CFE7
:1004A00006F0E4CF05F0E4CF04F0E4CF03F0E4CFAE
:1004B00002F0E4CF01F0E4CF00F0E4CFD9FF120066
:1004C000D9CFE5FFE1CFD9FF00C0E5FF01C0E5FFCF
:1004D00002C0E5FF03C0E5FF04C0E5FF05C0E5FF7E
:1004E00006C0E5FF07C0E5FF08C0E5FF020EDBCF51
:1004F00000F0030EDBCF01F0040EDBCF02F0050E9F
:10050000DBCF03F0060EDBCF04F0070EDBCF05F0E8
:10051000080EDBCF06F0090EDBCF07F0FAEC09F08E
:1005200003A003D0020EC86E02D0090EC86E36ECCE
:100530000BF00050E56EE3EC0AF0E12A03A208D0CC
:100540000250036E086A0350E56EE3EC0AF0E12AFC
:100550000150E56EE3EC0AF0E12A30EC0BF000808C
:100560000050E56EE3EC0AF0E12A04C000F005C09B
:1005700001F006C002F007C003F0020E035C16E3B0
:10058000010EE56E49EC0AF0046EE12A04C0E5FFB5
:1005900000C0E9FF01C0F3FF0250FBEC0AF0002AA3
:1005A000D8B0012AD8B0022A0306E7D703500FE0DB
:1005B000000EE56E49EC0AF0036EE12A03C0E5FF88
:1005C00000C0E9FF01C0F3FF0250FBEC0AF02AEC87
:1005D0000BF0E86AE4CF08F0E4CF07F0E4CF06F0D0
:1005E000E4CF05F0E4CF04F0E4CF03F0E4CF02F071
:1005F000E4CF01F0E4CF00F0E4CFD9FF1200620EA7
:10060000D36EFF0E926E0F0E936EFF0E946E816A84
:10061000D4EC0AF063EC09F00001806B816B826B13
:10062000030E836F010E846F856F866B100E876FCC
:10063000000E016E800E006E800E026E080EE56EDA
:100640000250E56E0150E56E0050E56E010EE56E5C
:10065000000EE56E000EE56ED00EE56E21EC04F0A6
:10066000080EE126030EE56EE80EE56ECBEC09F010
:10067000020EE126000E016E800E006E800E026EEC
:10068000080EE56E0250E56E0150E56E0050E56E15
:10069000000EE56E000EE56E000EE56ED00EE56E06
:1006A00060EC02F0080EE126000EE56E130EE56E1A
:1006B000F20EE56E000EE56E000EE56EA2EC04F0A3
:1006C000050EE12600018051E56E2EEC06F0E12AD0
:1006D00000018151E56E2EEC06F0E12A0001825105
:1006E000E56E2EEC06F0E12A00018351E56E2EEC5A
:1006F00006F0E12A00018451E56E2EEC06F0E12AB5
:1007000000018551E56E2EEC06F0E12A00018651CC
:10071000E56E2EEC06F0E12A00018751E56E2EEC25
:1007200006F0E12A9FD71200D9CFE5FFE1CFD9FF2C
:1007300000C0E5FF01C0E5FF02C0E5FF03C0E5FF23
:1007400004C0E5FF05C0E5FF06C0E5FF07C0E5FF03
:1007500008C0E5FF09C0E5FF0AC0E5FF0BC0E5FFE3
:100760000CC0E5FF0DC0E5FF020EDBCF00F0030E6D
:10077000DBCF01F0040EDBCF02F0050EDBCF03F080
:10078000060EDBCF04F0070EDBCF05F0080EDBCF43
:1007900006F0090EDBCF07F0086A096A0A6A0B6ADD
:1007A000200E0C6E0344010B0D6E010E0D16005051
:1007B00000260136023603360850082609360A3666
:1007C0000B360D50D8A4088007500B5C08E106508A
:1007D0000A5C05E10550095C02E10450085C09E38C
:1007E0000450085E0550095A06500A5A07500B5A21
:1007F00000800C2ED7D703C0E9FF02C0F4FF01C070
:10080000F3FF0050E4CF0DF0E4CF0CF0E4CF0BF099
:10081000E4CF0AF0E4CF09F0E4CF08F0E4CF07F02A
:10082000E4CF06F0E4CF05F0E4CF04F0E4CF03F02A
:10083000E4CF02F0E4CF01F0E4CF00F0E4CFD9FF41
:100840001200D9CFE5FFE1CFD9FF00C0E5FF01C01D
:10085000E5FF02C0E5FF03C0E5FF04C0E5FF05C0FA
:10086000E5FF06C0E5FF07C0E5FF020EDBCF00F0A5
:10087000030EDBCF01F0040EDBCF02F0050EDBCF61
:1008800003F0060EDBCF04F0070EDBCF05F0080EF9
:10089000DBCF06F0090EDBCF07F0FAEC09F003A07E
:1008A00003D0020EC86E02D0090EC86E36EC0BF0F3
:1008B0000050E56EE3EC0AF0E12A03A208D00250F2
:1008C000006E036A0050E56EE3EC0AF0E12A015085
:1008D000E56EE3EC0AF0E12A04C000F005C001F087
:1008E00006C002F007C003F003C004F00306045082
:1008F00013E000C0E9FF01C0F3FF0250A4EC0AF0CE
:10090000046E002AD8B0012AD8B0022A0450E56E3D
:10091000E3EC0AF0E12AE8D72AEC0BF0E86AE4CF2E
:1009200007F0E4CF06F0E4CF05F0E4CF04F0E4CF25
:1009300003F0E4CF02F0E4CF01F0E4CF00F0E4CF25
:10094000D9FF1200D9CFE5FFE1CFD9FF00C0E5FF05
:1009500001C0E5FF02C0E5FF03C0E5FF04C0E5FFFD
:10096000020EDBCF00F0030EDBCF01F0040EDBCF75
:1009700002F0050EDBCF03F0060EDBCF04F0FAEC3D
:1009800009F0090EC86E36EC0BF0C60EE56EE3EC0E
:100990000AF0E12A000EE56EE3EC0AF0E12AFE0E11
:1009A000E56EE3EC0AF0E12A0150400DF3CF01F0CF
:1009B000800E0126015000260050E56EE3EC0AF09F
:1009C000E12A02C000F003C001F004C002F000C040
:1009D000E9FF01C0F3FF0250A4EC0AF0036E0350DC
:1009E0000BE0002AD8B0012AD8B0022A0350E56EE5
:1009F000E3EC0AF0E12AEBD7FF0EE56EE3EC0AF038
:100A0000E12A2AEC0BF0000EE56E0A0EE56ECBEC47
:100A100009F0020EE126E4CF04F0E4CF03F0E4CFC6
:100A200002F0E4CF01F0E4CF00F0E4CFD9FF1200F0
:100A3000D9CFE5FFE1CFD9FF00C0E5FF01C0E5FF59
:100A400002C0E5FF03C0E5FF04C0E5FF05C0E5FF08
:100A500006C0E5FF07C0E5FF08C0E5FF09C0E5FFE8
:100A60000AC0E5FF0BC0E5FF020EDBCF00F000502F
:100A7000E56ED8EC07F0016EF3CF02F0E12A036ACD
:100A8000046A002A002A0050E56ED8EC07F0006ED8
:100A9000F3CF05F0E12A066A076A05500B6E005095
:100AA0000A6E086A096A08500112095002120A50B7
:100AB00003120B50041204C0E9FF03C0F4FF02C08C
:100AC000F3FF0150E4CF0BF0E4CF0AF0E4CF09F0DC
:100AD000E4CF08F0E4CF07F0E4CF06F0E4CF05F070
:100AE000E4CF04F0E4CF03F0E4CF02F0E4CF01F070
:100AF000E4CF00F0E4CFD9FF1200D9CFE5FFE1CF7A
:100B0000D9FF00C0E5FF01C0E5FF02C0E5FF03C05B
:100B1000E5FF04C0E5FF05C0E5FF06C0E5FF020EE6
:100B2000DBCF00F0030EDBCF01F0040EDBCF02F0D1
:100B3000050EDBCF03F0046A056A0344010B066E61
:100B400006B011D00250022603360350015C02E1C8
:100B50000250005C04E2D8900332023204D0052A2D
:100B600005C004F0EAD70350015C02E10250005CCA
:100B700004E30250005E0350015AD890033202325F
:100B800004C005F004060550EEE101C0F3FF00507B
:100B9000E4CF06F0E4CF05F0E4CF04F0E4CF03F0B7
:100BA000E4CF02F0E4CF01F0E4CF00F0E4CFD9FFCE
:100BB0001200D9CFE5FFE1CFD9FF00C0E5FF01C0AA
:100BC000E5FF02C0E5FF03C0E5FF04C0E5FF05C087
:100BD000E5FF06C0E5FF07C0E5FF020EDBCF00F032
:100BE000030EDBCF01F0040EDBCF02F0050EDBCFEE
:100BF00003F0046A056A100E066E0144010B076ECD
:100C0000010E071600500026013604500426053652
:100C10000750D8A404800350055C02E10250045C34
:100C200005E30250045E0350055A0080062EE5D706
:100C300001C0F3FF0050E4CF07F0E4CF06F0E4CFAB
:100C400005F0E4CF04F0E4CF03F0E4CF02F0E4CF0A
:100C500001F0E4CF00F0E4CFD9FF1200D9CFE5FFD7
:100C6000E1CFD9FF00C0E5FF01C0E5FF02C0E5FF0D
:100C7000020EDBCF00F000380F0B016E300E0126A4
:100C80003A0E015C02E3070E012601500001936F4A
:100C90000F0E0014016E300E01263A0E015C02E3C5
:100CA000070E012601500001946F9569000E016E38
:100CB000930E006E800E026E030EE56E0250E56E1E
:100CC0000150E56E0050E56E000EE56E000EE56E1B
:100CD000000EE56EC60EE56E21EC04F0080EE1266E
:100CE000000EE56E0A0EE56ECBEC09F0020EE12671
:100CF000E4CF02F0E4CF01F0E4CF00F0E4CFD9FF7D
:100D00001200D9CFE5FFE1CFD9FF00C0E5FF01C058
:100D1000E5FF02C0E5FF03C0E5FF04C0E5FF05C035
:100D2000E5FF06C0E5FF020EDBCF00F0030EDBCFD0
:100D300001F0040EDBCF02F0050EDBCF03F0060E50
:100D4000DBCF04F00150056E0250066EE56E0550D3
:100D5000E56E0050E56E9DEC07F0030EE126002ADB
:100D6000002A0350016E0450026E036A046A0250A6
:100D7000E56E0150E56E0050E56E9DEC07F0030E48
:100D8000E126E4CF06F0E4CF05F0E4CF04F0E4CFB1
:100D900003F0E4CF02F0E4CF01F0E4CF00F0E4CFC1
:100DA000D9FF12003A0EF66E160EF76E000EF86EB0
:100DB0000900F550056E0900F550066E055002E178
:100DC00006503BE00900F550006E0900F550016E39
:100DD0000900F550026E09000900F550E96E09009E
:100DE000F550EA6E090009000900F550036E09008C
:100DF000F550046E09000900F6CF07F0F7CF08F0B0
:100E0000F8CF09F000C0F6FF01C0F7FF02C0F8FFFD
:100E1000035002E1045007E00900F550EE6E0306AE
:100E2000F8E20406F9D707C0F6FF08C0F7FF09C0CB
:100E3000F8FF0506C4E20606C5D71200D9CFE5FFC4
:100E4000E1CFD9FF00C0E5FF01C0E5FF02C0E5FF2B
:100E500003C0E5FF04C0E5FF05C0E5FF020EDBCFE0
:100E600000F0030EDBCF01F0040EDBCF02F0050E25
:100E7000DBCF03F0046A0350045C14E200C0E9FF16
:100E800001C0F3FF0250A4EC0AF0056E002AD8B0AE
:100E9000012AD8B0022A0550E56E92EC0AF0E12A48
:100EA000042AE9D7E4CF05F0E4CF04F0E4CF03F05F
:100EB000E4CF02F0E4CF01F0E4CF00F0E4CFD9FFBB
:100EC0001200D9CFE5FFE1CFD9FF00C0E5FF01C097
:100ED000E5FF02C0E5FF020EDBCF00F0005000018D
:100EE000966F9769000E016E960E006E800E026E70
:100EF000020EE56E0250E56E0150E56E0050E56EA3
:100F0000000EE56E000EE56E000EE56EC60EE56E97
:100F100021EC04F0080EE126000EE56E0A0EE56EE7
:100F2000CBEC09F0020EE126E4CF02F0E4CF01F0B1
:100F3000E4CF00F0E4CFD9FF1200D9CFE5FFE1CF35
:100F4000D9FF00C0E5FF01C0E5FF02C0E5FF020ECA
:100F5000DBCF00F0030EDBCF01F0040EDBCF02F09D
:100F6000A69EA69CA684F29E00C0A9FF0150A86E72
:100F7000550EA76EAA0EA76EA682A6B2FED70028AF
:100F8000A96E0250016E026A0150A86E550EA76E3E
:100F9000AA0EA76EA682A6B2FED7A694F28EE4CFC2
:100FA00002F0E4CF01F0E4CF00F0E4CFD9FF12006B
:100FB000D9CFE5FFE1CFD9FF00C0E5FF01C0E5FFD4
:100FC00002C0E5FF03C0E5FF04C0E5FF05C0E5FF83
:100FD000020EDBCF00F0A69CA69E00C0A9FFA68053
:100FE000A8CF01F0026A0028A96EA680A8CF00F061
:100FF000036A0050056E046A045001120550021283
:1010000002C0F3FF0150E4CF05F0E4CF04F0E4CFD9
:1010100003F0E4CF02F0E4CF01F0E4CF00F0E4CF3E
:10102000D9FF1200D9CFE5FFE1CFD9FF00C0E5FF1E
:1010300001C0E5FF02C0E5FF03C0E5FF020EDBCF04
:1010400000F0030EDBCF01F0040EDBCF02F000C096
:10105000E9FF01C0F3FF0250A4EC0AF0036E035055
:1010600010E0ACA2FED700C0E9FF01C0F3FF0250C0
:10107000A4EC0AF0AD6E002AD8B0012AD8B0022A3A
:10108000E6D7E4CF03F0E4CF02F0E4CF01F0E4CF01
:1010900000F0E4CFD9FF1200D9CFE5FFE1CFD9FFAF
:1010A00000C0E5FF01C0E5FF02C0E5FF03C0E5FFAA
:1010B000020EDBCF00F0030EDBCF01F0026A036A01
:1010C00001BE0CD0D89001360150005C03E2D890EC
:1010D000013204D0032A03C002F0F2D70150005CB1
:1010E00002E30150005ED890013202C003F0020614
:1010F0000350F4E10050E4CF03F0E4CF02F0E4CF7A
:1011000001F0E4CF00F0E4CFD9FF120000C0E5FF0A
:1011100001C0E5FF02C0E5FF03C0E5FF2DEC09F0CB
:10112000006EF3CF01F0F4CF02F0E9CF03F0000E30
:10113000E56E0F0EE56E420EE56E400EE56E035055
:10114000E56E0250E56E0150E56E0050E56E94ECE0
:1011500003F0006EF3CF01F0F4CF02F0E9CF03F01B
:10116000080EE12601C0F3FF0050E4CF03F0E4CF06
:1011700002F0E4CF01F0E4CF00F0120000C0E5FF80
:1011800001C0E5FF02C0E5FF03C0E5FF2DEC09F05B
:10119000006EF3CF01F0F4CF02F0E9CF03F0000EC0
:1011A000E56E000EE56E030EE56EE80EE56E03508B
:1011B000E56E0250E56E0150E56E0050E56E94EC70
:1011C00003F0006EF3CF01F0F4CF02F0E9CF03F0AB
:1011D000080EE12601C0F3FF0050E4CF03F0E4CF96
:1011E00002F0E4CF01F0E4CF00F01200D9CFE5FF28
:1011F000E1CFD9FF00C0E5FF01C0E5FF02C0E5FF78
:1012000003C0E5FF04C0E5FF020EDBCF00F0030ED4
:10121000DBCF01F0026A080E036E800E0014046E2C
:10122000D8900036D89002360450D8A402800150DD
:10123000025C03E30150025E0080032EEED70050F3
:10124000E4CF04F0E4CF03F0E4CF02F0E4CF01F008
:10125000E4CF00F0E4CFD9FF120000C0E5FF01C0E9
:10126000E5FF02C0E5FF03C0E5FF04C0E5FF05C0E0
:10127000E5FFB2CF00F0B3CF01F098C002F099C003
:1012800003F0B2CF04F0B3CF05F00150055C02E1EA
:101290000050045C04E298C002F099C003F003C05F
:1012A000E9FF02C0F4FF05C0F3FF0450E4CF05F0EE
:1012B000E4CF04F0E4CF03F0E4CF02F0E4CF01F098
:1012C000E4CF00F0120000C0E5FF01C0E5FF02C05E
:1012D000E5FFFE0E0001906F010E916F9269000E06
:1012E000016E900E006E800E026E030EE56E0250CF
:1012F000E56E0150E56E0050E56E000EE56E000EE5
:10130000E56E000EE56EC60EE56E21EC04F0080EEB
:10131000E126000EE56E0A0EE56ECBEC09F0020E3A
:10132000E126E4CF02F0E4CF01F0E4CF00F01200B8
:10133000D9CFE5FFE1CFD9FF00C0E5FF01C0E5FF50
:1013400002C0E5FF03C0E5FF020EDBCF00F0004462
:10135000E844FC0B016E030E0110C26EC2B2FED750
:10136000C4CF00F0016A0050036E026AC3CF00F0E0
:10137000016A005002260150032203C0F3FF02500D
:10138000E4CF03F0E4CF02F0E4CF01F0E4CF00F0CB
:10139000E4CFD9FF1200D9CFE5FFE1CFD9FF00C0DC
:1013A000E5FF01C0E5FF02C0E5FF03C0E5FF020E57
:1013B000DBCF00F0030EDBCF01F000C002F001C074
:1013C00003F0FF0E0026D8A001060250031006E02D
:1013D000FA0E026E0000022EFDD7EFD7E4CF03F025
:1013E000E4CF02F0E4CF01F0E4CF00F0E4CFD9FF86
:1013F0001200000000C0E5FF01C0E5FF02C0E5FFEC
:10140000FF0E006E1F0EC514016E026AC7B4022AD9
:1014100002500112015003E000060050F3E100C049
:1014200001F00050D8B4B5EC0AF00150D880E8665D
:10143000D890016A01360150E4CF02F0E4CF01F008
:10144000E4CF00F01200D9CFE5FFE1CFD9FF00C013
:10145000E5FF01C0E5FF020EDBCF00F0030EDBCF9E
:1014600001F0A69EA69CA684F29E01C0A8FF00C023
:10147000A9FF550EA76EAA0EA76EA682A6B2FED72A
:10148000A694F28EE4CF01F0E4CF00F0E4CFD9FFD0
:101490001200D9CFE5FFE1CFD9FF00C0E5FF01C0C1
:1014A000E5FF020EDBCF00F0FAEC09F0C586FAEC9E
:1014B00009F0C9CF01F0FAEC09F0005002E0C59A3A
:1014C00001D0C58AC5880150E4CF01F0E4CF00F017
:1014D000E4CFD9FF1200D9CFE5FFE1CFD9FF00C09B
:1014E000E5FF020EDBCF00F0A69CA69E00C0A9FF80
:1014F000A680A850E4CF00F0E4CFD9FF120000C0CE
:10150000E5FF01C0E5FF1F0EC514006E016AC7B4F8
:10151000012A015000120050F6E1E4CF01F0E4CFBF
:1015200000F01200D9CFE5FFE1CFD9FF00C0E5FF01
:10153000020EDBCF00F0ACA2FED700C0ADFFE4CFBF
:1015400000F0E4CFD9FF1200E8AE04D0F3CFEAFFF9
:10155000EE501200E8BC08D0E9CFF6FFF3CFF7FF5A
:10156000F86E0900F55012001200818AC69A94960E
:10157000828682B803D082968286FBD7949882981E
:10158000828894869488C68A1200200EAC6E900ED3
:10159000AB6E0C0EAF6E000EE56E010EE56ECBEC81
:1015A00009F0020EE12612003F0EC716280EC66E85
:1015B000C56A090EC86E948694889E96A196B5EC6D
:1015C0000AF0819A1200D9CFE5FFE1CFD9FF020ED0
:1015D000DBCFC9FFFAEC09F0E4CFD9FF120012EE1D
:1015E000FFF022EEFFF0F86AA68EA69CD2EC06F081
:1015F000FFEC02F0FFD7E8AE05D0F3CFEAFFE4CF6F
:10160000EEFF1200E8AC1200120000C0E5FF006A15
:101610009EBA002A0050E4CF00F01200810EB16E95
:10162000B36AB26A0001986B996B1200010EC26E28
:10163000050EC16E940EC06E120001008A160000E5
:101640009A00000001000000B36AB26A0001986BC2
:10165000996B1200FAEC09F0C584C5B4FED71200EC
:10166000FAEC09F0C582C5B2FED71200FAEC09F017
:10167000C580C5B0FED712000001982B01E3992B5D
:0C16800012009EAAFED7AE50120000001F
:00000001FF
